:02000000800B73
:10000B002167758129758902758C2275A8827525E2
:10001B0000752600752240752700752800E590F4C1
:10002B0054E0F521D2B5C2B1D2B211FBD2B4D28C0D
:10003B00E525B40CFB752500E590F4541FB524F0B1
:10004B00E523A200B0024050A202B000404AB41017
:10005B000DE521B4FF02803A052111FB8034B41168
:10006B000AE521602D152111FB8027B41A028003AC
:10007B00B4340DE522B480028018052211FB8012E6
:10008B00B41B028003B4320AE5226006152211FB71
:10009B008000A20092028098F5F014C39408501DC2
:1000AB00E5F0C394075009E5F014F52711FB80E246
:1000BB00E5F01490022693622811FB80D5E5F0B48D
:1000CB000C04B2B480CCB40D04B2B580C5B4200E10
:1000DB00E527B405037527FF052711FB80B4B42171
:1000EB000DE5277003752706152711FB80A4015911
:1000FB00C2B2E5217B10C34002940F3150DBF8E50F
:10010B0022B44004D2B38002C2B3C39440500DABAF
:10011B0021E5228521F03159ACF0800EAC217480A1
:10012B00C395228521F03159ABF0EC3148EB3148C6
:10013B00E5279002269345283148D2B2227A08331C
:10014B003150DAFB2292B000D2B100C2B122A433FB
:10015B00C5F033C5F033C5F033C5F022C0E0C0D0D5
:10016B00C082C0839001C0A2B7B3E5263393F526B6
:10017B00B4210B752500752400752300802EB42A3D
:10018B0004D2018005B43224C2010525E525B40152
:10019B0006A20192008015C394075009A201E52421
:1001AB0033F5248007A201E52333F523D083D082D6
:1001BB00D0D0D0E03201000200030004000500069D
:1001CB00000700080009000A000B000C000D000ED0
:1001DB00000F001000110012001300140014150082
:1001EB001600171A181A191A001B001C001D1F1EC7
:1001FB001F001F002000212322232B242B25002648
:10020B0028272800280029002A2322232C002D3000
:10021B002E302F300031003200222B010204081047
:03022B00204080F0
:00000001FF
